MPLINK 4.40, Linker
Linker Map File - Created Tue Feb 07 01:02:51 2012

                                 Section Info
                  Section       Type    Address   Location Size(Bytes)
                ---------  ---------  ---------  ---------  ---------
               _entry_scn       code   0x000000    program   0x000006
                   .cinit    romdata   0x00002a    program   0x00000e
         .code_enc28j60.o       code   0x000038    program   0x000c62
               .code_ip.o       code   0x000c9a    program   0x0003f2
              .code_arp.o       code   0x00108c    program   0x0001d2
             .code_icmp.o       code   0x00125e    program   0x000118
            .code_stack.o       code   0x001376    program   0x0000a6
               _cinit_scn       code   0x00141c    program   0x00009e
          .code_utility.o       code   0x0014ba    program   0x00004a
                    .code       code   0x001504    program   0x000020
             _startup_scn       code   0x001524    program   0x00001c
             D100TCYXCODE       code   0x001540    program   0x00001c
             .code_main.o       code   0x00155c    program   0x00000c
           .code___init.o       code   0x001568    program   0x000002
          .romdata_icmp.o    romdata   0x00156a    program   0x000000
           .romdata_arp.o    romdata   0x00156a    program   0x000000
         .romdata_c018i.o    romdata   0x00156a    program   0x000000
            .romdata_ip.o    romdata   0x00156a    program   0x000000
            .idata_ip.o_i    romdata   0x00156a    program   0x000002
          .idata_main.o_i    romdata   0x00156a    program   0x000000
         .romdata_stack.o    romdata   0x00156a    program   0x000000
         .idata_stack.o_i    romdata   0x00156a    program   0x000000
          .romdata_main.o    romdata   0x00156a    program   0x000000
       .romdata_utility.o    romdata   0x00156a    program   0x000000
       .idata_utility.o_i    romdata   0x00156a    program   0x000000
      .romdata_enc28j60.o    romdata   0x00156a    program   0x000000
        .romdata___init.o    romdata   0x00156a    program   0x000000
        .idata___init.o_i    romdata   0x00156c    program   0x000000
         .idata_c018i.o_i    romdata   0x00156c    program   0x000000
          .idata_icmp.o_i    romdata   0x00156c    program   0x000000
            .code_c018i.o       code   0x00156c    program   0x000000
           .idata_arp.o_i    romdata   0x00156c    program   0x000000
      .idata_enc28j60.o_i    romdata   0x00156c    program   0x000000
    .config_300001_main.o    romdata   0x300001    program   0x000001
    .config_300002_main.o    romdata   0x300002    program   0x000001
    .config_300003_main.o    romdata   0x300003    program   0x000001
    .config_300005_main.o    romdata   0x300005    program   0x000001
    .config_300006_main.o    romdata   0x300006    program   0x000001
                MATH_DATA      udata   0x000000       data   0x00000b
                 .tmpdata      udata   0x00000b       data   0x000006
                DELAYDAT1      udata   0x000011       data   0x000001
           .udata_c018i.o      udata   0x000080       data   0x00000a
           .udata_stack.o      udata   0x00008a       data   0x000006
        .udata_enc28j60.o      udata   0x000090       data   0x000006
              .udata_ip.o      udata   0x000096       data   0x000004
              .idata_ip.o      idata   0x00009a       data   0x000002
          .idata___init.o      idata   0x00009c       data   0x000000
          .udata___init.o      udata   0x00009c       data   0x000000
            .idata_icmp.o      idata   0x00009c       data   0x000000
            .udata_icmp.o      udata   0x00009c       data   0x000000
             .idata_arp.o      idata   0x00009c       data   0x000000
             .udata_arp.o      udata   0x00009c       data   0x000000
           .idata_stack.o      idata   0x00009c       data   0x000000
         .idata_utility.o      idata   0x00009c       data   0x000000
         .udata_utility.o      udata   0x00009c       data   0x000000
        .idata_enc28j60.o      idata   0x00009c       data   0x000000
            .idata_main.o      idata   0x00009c       data   0x000000
            .udata_main.o      udata   0x00009c       data   0x000000
           .idata_c018i.o      idata   0x00009c       data   0x000000
                   .stack      udata   0x000e00       data   0x000100
            SFR_UNBANKED0      udata   0x000f80       data   0x000080



                              Program Memory Usage 
                               Start         End      
                           ---------   ---------      
                            0x000000    0x000005      
                            0x00002a    0x00156b      
                            0x300001    0x300003      
                            0x300005    0x300006      
            5453 out of 66584 program addresses used, program memory utilization is 8%



                              Symbols - Sorted by Name
                     Name    Address   Location    Storage File                     
                ---------  ---------  ---------  --------- ---------                
                   BFCReg   0x000bf8    program     extern C:\Documents and Settings\User\Desktop\RFID Ethernet\Seconda Parte\Interfaccia Ethernet con ENC28J60\02_icmp_C18\enc28j60.c
                   BFSReg   0x000c22    program     extern C:\Documents and Settings\User\Desktop\RFID Ethernet\Seconda Parte\Interfaccia Ethernet con ENC28J60\02_icmp_C18\enc28j60.c
                   D100_1   0x00154e    program     static C:\MCC18\v3_39\src\traditional\delays\d100tcyx.asm
                    D100x   0x00154c    program     static C:\MCC18\v3_39\src\traditional\delays\d100tcyx.asm
              DMAChecksum   0x000246    program     extern C:\Documents and Settings\User\Desktop\RFID Ethernet\Seconda Parte\Interfaccia Ethernet con ENC28J60\02_icmp_C18\enc28j60.c
             Delay100TCYx   0x001540    program     extern C:\MCC18\v3_39\src\traditional\delays\d100tcyx.asm
              IPPutHeader   0x000f1a    program     extern C:\Documents and Settings\User\Desktop\RFID Ethernet\Seconda Parte\Interfaccia Ethernet con ENC28J60\02_icmp_C18\ip.c
             MACGetHeader   0x0005d6    program     extern C:\Documents and Settings\User\Desktop\RFID Ethernet\Seconda Parte\Interfaccia Ethernet con ENC28J60\02_icmp_C18\enc28j60.c
             MACPutHeader   0x000764    program     extern C:\Documents and Settings\User\Desktop\RFID Ethernet\Seconda Parte\Interfaccia Ethernet con ENC28J60\02_icmp_C18\enc28j60.c
                  MACSend   0x000842    program     extern C:\Documents and Settings\User\Desktop\RFID Ethernet\Seconda Parte\Interfaccia Ethernet con ENC28J60\02_icmp_C18\enc28j60.c
       _D100TCYXCODE_0008   0x001548    program     static C:\MCC18\v3_39\src\traditional\delays\d100tcyx.asm
       _D100TCYXCODE_0012   0x001552    program     static C:\MCC18\v3_39\src\traditional\delays\d100tcyx.asm
       _D100TCYXCODE_0018   0x001558    program     static C:\MCC18\v3_39\src\traditional\delays\d100tcyx.asm
       ___return_lbl00000   0x000004    program     static                          
       ___return_lbl00001   0x00153e    program     static                          
       ___return_lbl00002   0x0014b8    program     static                          
               __config_0   0x300001    program     static C:\Documents and Settings\User\Desktop\RFID Ethernet\Seconda Parte\Interfaccia Ethernet con ENC28J60\02_icmp_C18\main.c
               __config_1   0x300002    program     static C:\Documents and Settings\User\Desktop\RFID Ethernet\Seconda Parte\Interfaccia Ethernet con ENC28J60\02_icmp_C18\main.c
               __config_2   0x300003    program     static C:\Documents and Settings\User\Desktop\RFID Ethernet\Seconda Parte\Interfaccia Ethernet con ENC28J60\02_icmp_C18\main.c
               __config_3   0x300005    program     static C:\Documents and Settings\User\Desktop\RFID Ethernet\Seconda Parte\Interfaccia Ethernet con ENC28J60\02_icmp_C18\main.c
               __config_4   0x300006    program     static C:\Documents and Settings\User\Desktop\RFID Ethernet\Seconda Parte\Interfaccia Ethernet con ENC28J60\02_icmp_C18\main.c
                   __init   0x001568    program     extern C:\MCC18\v3_39\src\traditional\stdclib\__init.c
            __zero_memory   0x001504    program     extern C:\MCC18\v3_39\src\traditional\proc\p18F2620.asm
                _do_cinit   0x00141c    program     extern C:\MCC18\v3_39\src\traditional\startup\c018i.c
                   _entry   0x000000    program     extern C:\MCC18\v3_39\src\traditional\startup\c018i.c
                 _startup   0x001524    program     extern C:\MCC18\v3_39\src\traditional\startup\c018i.c
                compare_l   0x00151a    program     static C:\MCC18\v3_39\src\traditional\proc\p18F2620.asm
                copy_loop   0x00148e    program     static                          
            copy_one_byte   0x001494    program     static                          
                     done   0x0014b8    program     static                          
             done_copying   0x0014a2    program     static                          
               encDiscard   0x000536    program     extern C:\Documents and Settings\User\Desktop\RFID Ethernet\Seconda Parte\Interfaccia Ethernet con ENC28J60\02_icmp_C18\enc28j60.c
                   encGet   0x000a22    program     extern C:\Documents and Settings\User\Desktop\RFID Ethernet\Seconda Parte\Interfaccia Ethernet con ENC28J60\02_icmp_C18\enc28j60.c
              encGetArray   0x0008e4    program     extern C:\Documents and Settings\User\Desktop\RFID Ethernet\Seconda Parte\Interfaccia Ethernet con ENC28J60\02_icmp_C18\enc28j60.c
                  encInit   0x000038    program     extern C:\Documents and Settings\User\Desktop\RFID Ethernet\Seconda Parte\Interfaccia Ethernet con ENC28J60\02_icmp_C18\enc28j60.c
                   encPut   0x0009f4    program     extern C:\Documents and Settings\User\Desktop\RFID Ethernet\Seconda Parte\Interfaccia Ethernet con ENC28J60\02_icmp_C18\enc28j60.c
              encPutArray   0x00093a    program     extern C:\Documents and Settings\User\Desktop\RFID Ethernet\Seconda Parte\Interfaccia Ethernet con ENC28J60\02_icmp_C18\enc28j60.c
             encPutString   0x0009a0    program     extern C:\Documents and Settings\User\Desktop\RFID Ethernet\Seconda Parte\Interfaccia Ethernet con ENC28J60\02_icmp_C18\enc28j60.c
              freeRxSpace   0x0006ba    program     extern C:\Documents and Settings\User\Desktop\RFID Ethernet\Seconda Parte\Interfaccia Ethernet con ENC28J60\02_icmp_C18\enc28j60.c
                    htons   0x0014ba    program     extern C:\Documents and Settings\User\Desktop\RFID Ethernet\Seconda Parte\Interfaccia Ethernet con ENC28J60\02_icmp_C18\utility.c
                  ipMatch   0x000c9a    program     extern C:\Documents and Settings\User\Desktop\RFID Ethernet\Seconda Parte\Interfaccia Ethernet con ENC28J60\02_icmp_C18\ip.c
              isMACLinked   0x0008cc    program     extern C:\Documents and Settings\User\Desktop\RFID Ethernet\Seconda Parte\Interfaccia Ethernet con ENC28J60\02_icmp_C18\enc28j60.c
                     loop   0x001534    program     static                          
                   loop_h   0x001512    program     static C:\MCC18\v3_39\src\traditional\proc\p18F2620.asm
                   loop_l   0x00151c    program     static C:\MCC18\v3_39\src\traditional\proc\p18F2620.asm
                     main   0x00155c    program     extern C:\Documents and Settings\User\Desktop\RFID Ethernet\Seconda Parte\Interfaccia Ethernet con ENC28J60\02_icmp_C18\main.c
               processARP   0x00108c    program     extern C:\Documents and Settings\User\Desktop\RFID Ethernet\Seconda Parte\Interfaccia Ethernet con ENC28J60\02_icmp_C18\arp.c
              processICMP   0x00125e    program     extern C:\Documents and Settings\User\Desktop\RFID Ethernet\Seconda Parte\Interfaccia Ethernet con ENC28J60\02_icmp_C18\icmp.c
                processIP   0x000dd2    program     extern C:\Documents and Settings\User\Desktop\RFID Ethernet\Seconda Parte\Interfaccia Ethernet con ENC28J60\02_icmp_C18\ip.c
            processPacket   0x001376    program     extern C:\Documents and Settings\User\Desktop\RFID Ethernet\Seconda Parte\Interfaccia Ethernet con ENC28J60\02_icmp_C18\stack.c
              putChecksum   0x000422    program     extern C:\Documents and Settings\User\Desktop\RFID Ethernet\Seconda Parte\Interfaccia Ethernet con ENC28J60\02_icmp_C18\enc28j60.c
                  readETH   0x000bca    program     extern C:\Documents and Settings\User\Desktop\RFID Ethernet\Seconda Parte\Interfaccia Ethernet con ENC28J60\02_icmp_C18\enc28j60.c
                  readMAC   0x000b96    program     extern C:\Documents and Settings\User\Desktop\RFID Ethernet\Seconda Parte\Interfaccia Ethernet con ENC28J60\02_icmp_C18\enc28j60.c
                  readPHY   0x000b06    program     extern C:\Documents and Settings\User\Desktop\RFID Ethernet\Seconda Parte\Interfaccia Ethernet con ENC28J60\02_icmp_C18\enc28j60.c
                sendReset   0x000a4e    program     extern C:\Documents and Settings\User\Desktop\RFID Ethernet\Seconda Parte\Interfaccia Ethernet con ENC28J60\02_icmp_C18\enc28j60.c
                  setBank   0x000c4c    program     extern C:\Documents and Settings\User\Desktop\RFID Ethernet\Seconda Parte\Interfaccia Ethernet con ENC28J60\02_icmp_C18\enc28j60.c
                    spiRW   0x000c7a    program     extern C:\Documents and Settings\User\Desktop\RFID Ethernet\Seconda Parte\Interfaccia Ethernet con ENC28J60\02_icmp_C18\enc28j60.c
             swapIPHeader   0x000cea    program     extern C:\Documents and Settings\User\Desktop\RFID Ethernet\Seconda Parte\Interfaccia Ethernet con ENC28J60\02_icmp_C18\ip.c
                     test   0x001436    program     static                          
                 writePHY   0x000a84    program     extern C:\Documents and Settings\User\Desktop\RFID Ethernet\Seconda Parte\Interfaccia Ethernet con ENC28J60\02_icmp_C18\enc28j60.c
                 writeReg   0x000a5a    program     extern C:\Documents and Settings\User\Desktop\RFID Ethernet\Seconda Parte\Interfaccia Ethernet con ENC28J60\02_icmp_C18\enc28j60.c
               zero_block   0x001512    program     static C:\MCC18\v3_39\src\traditional\proc\p18F2620.asm
                   ADCON0   0x000fc2       data     extern C:\MCC18\v3_39\src\traditional\proc\p18F2620.asm
               ADCON0bits   0x000fc2       data     extern C:\MCC18\v3_39\src\traditional\proc\p18F2620.asm
                   ADCON1   0x000fc1       data     extern C:\MCC18\v3_39\src\traditional\proc\p18F2620.asm
               ADCON1bits   0x000fc1       data     extern C:\MCC18\v3_39\src\traditional\proc\p18F2620.asm
                   ADCON2   0x000fc0       data     extern C:\MCC18\v3_39\src\traditional\proc\p18F2620.asm
               ADCON2bits   0x000fc0       data     extern C:\MCC18\v3_39\src\traditional\proc\p18F2620.asm
                    ADRES   0x000fc3       data     extern C:\MCC18\v3_39\src\traditional\proc\p18F2620.asm
                   ADRESH   0x000fc4       data     extern C:\MCC18\v3_39\src\traditional\proc\p18F2620.asm
                   ADRESL   0x000fc3       data     extern C:\MCC18\v3_39\src\traditional\proc\p18F2620.asm
                  BAUDCON   0x000fb8       data     extern C:\MCC18\v3_39\src\traditional\proc\p18F2620.asm
              BAUDCONbits   0x000fb8       data     extern C:\MCC18\v3_39\src\traditional\proc\p18F2620.asm
                  BAUDCTL   0x000fb8       data     extern C:\MCC18\v3_39\src\traditional\proc\p18F2620.asm
              BAUDCTLbits   0x000fb8       data     extern C:\MCC18\v3_39\src\traditional\proc\p18F2620.asm
                      BSR   0x000fe0       data     extern C:\MCC18\v3_39\src\traditional\proc\p18F2620.asm
                  CCP1CON   0x000fbd       data     extern C:\MCC18\v3_39\src\traditional\proc\p18F2620.asm
              CCP1CONbits   0x000fbd       data     extern C:\MCC18\v3_39\src\traditional\proc\p18F2620.asm
                  CCP2CON   0x000fba       data     extern C:\MCC18\v3_39\src\traditional\proc\p18F2620.asm
              CCP2CONbits   0x000fba       data     extern C:\MCC18\v3_39\src\traditional\proc\p18F2620.asm
                    CCPR1   0x000fbe       data     extern C:\MCC18\v3_39\src\traditional\proc\p18F2620.asm
                   CCPR1H   0x000fbf       data     extern C:\MCC18\v3_39\src\traditional\proc\p18F2620.asm
                   CCPR1L   0x000fbe       data     extern C:\MCC18\v3_39\src\traditional\proc\p18F2620.asm
                    CCPR2   0x000fbb       data     extern C:\MCC18\v3_39\src\traditional\proc\p18F2620.asm
                   CCPR2H   0x000fbc       data     extern C:\MCC18\v3_39\src\traditional\proc\p18F2620.asm
                   CCPR2L   0x000fbb       data     extern C:\MCC18\v3_39\src\traditional\proc\p18F2620.asm
                    CMCON   0x000fb4       data     extern C:\MCC18\v3_39\src\traditional\proc\p18F2620.asm
                CMCONbits   0x000fb4       data     extern C:\MCC18\v3_39\src\traditional\proc\p18F2620.asm
                   CVRCON   0x000fb5       data     extern C:\MCC18\v3_39\src\traditional\proc\p18F2620.asm
               CVRCONbits   0x000fb5       data     extern C:\MCC18\v3_39\src\traditional\proc\p18F2620.asm
                     DDRA   0x000f92       data     extern C:\MCC18\v3_39\src\traditional\proc\p18F2620.asm
                 DDRAbits   0x000f92       data     extern C:\MCC18\v3_39\src\traditional\proc\p18F2620.asm
                     DDRB   0x000f93       data     extern C:\MCC18\v3_39\src\traditional\proc\p18F2620.asm
                 DDRBbits   0x000f93       data     extern C:\MCC18\v3_39\src\traditional\proc\p18F2620.asm
                     DDRC   0x000f94       data     extern C:\MCC18\v3_39\src\traditional\proc\p18F2620.asm
                 DDRCbits   0x000f94       data     extern C:\MCC18\v3_39\src\traditional\proc\p18F2620.asm
            DelayCounter1   0x000011       data     extern C:\MCC18\v3_39\src\traditional\delays\delayd1.asm
                  ECCP1AS   0x000fb6       data     extern C:\MCC18\v3_39\src\traditional\proc\p18F2620.asm
              ECCP1ASbits   0x000fb6       data     extern C:\MCC18\v3_39\src\traditional\proc\p18F2620.asm
                 ECCP1DEL   0x000fb7       data     extern C:\MCC18\v3_39\src\traditional\proc\p18F2620.asm
             ECCP1DELbits   0x000fb7       data     extern C:\MCC18\v3_39\src\traditional\proc\p18F2620.asm
                   ECCPAS   0x000fb6       data     extern C:\MCC18\v3_39\src\traditional\proc\p18F2620.asm
               ECCPASbits   0x000fb6       data     extern C:\MCC18\v3_39\src\traditional\proc\p18F2620.asm
                    EEADR   0x000fa9       data     extern C:\MCC18\v3_39\src\traditional\proc\p18F2620.asm
                   EEADRH   0x000faa       data     extern C:\MCC18\v3_39\src\traditional\proc\p18F2620.asm
                   EECON1   0x000fa6       data     extern C:\MCC18\v3_39\src\traditional\proc\p18F2620.asm
               EECON1bits   0x000fa6       data     extern C:\MCC18\v3_39\src\traditional\proc\p18F2620.asm
                   EECON2   0x000fa7       data     extern C:\MCC18\v3_39\src\traditional\proc\p18F2620.asm
                   EEDATA   0x000fa8       data     extern C:\MCC18\v3_39\src\traditional\proc\p18F2620.asm
                     FSR0   0x000fe9       data     extern C:\MCC18\v3_39\src\traditional\proc\p18F2620.asm
                    FSR0H   0x000fea       data     extern C:\MCC18\v3_39\src\traditional\proc\p18F2620.asm
                    FSR0L   0x000fe9       data     extern C:\MCC18\v3_39\src\traditional\proc\p18F2620.asm
                     FSR1   0x000fe1       data     extern C:\MCC18\v3_39\src\traditional\proc\p18F2620.asm
                    FSR1H   0x000fe2       data     extern C:\MCC18\v3_39\src\traditional\proc\p18F2620.asm
                    FSR1L   0x000fe1       data     extern C:\MCC18\v3_39\src\traditional\proc\p18F2620.asm
                     FSR2   0x000fd9       data     extern C:\MCC18\v3_39\src\traditional\proc\p18F2620.asm
                    FSR2H   0x000fda       data     extern C:\MCC18\v3_39\src\traditional\proc\p18F2620.asm
                    FSR2L   0x000fd9       data     extern C:\MCC18\v3_39\src\traditional\proc\p18F2620.asm
                  HLVDCON   0x000fd2       data     extern C:\MCC18\v3_39\src\traditional\proc\p18F2620.asm
              HLVDCONbits   0x000fd2       data     extern C:\MCC18\v3_39\src\traditional\proc\p18F2620.asm
                    INDF0   0x000fef       data     extern C:\MCC18\v3_39\src\traditional\proc\p18F2620.asm
                    INDF1   0x000fe7       data     extern C:\MCC18\v3_39\src\traditional\proc\p18F2620.asm
                    INDF2   0x000fdf       data     extern C:\MCC18\v3_39\src\traditional\proc\p18F2620.asm
                   INTCON   0x000ff2       data     extern C:\MCC18\v3_39\src\traditional\proc\p18F2620.asm
                  INTCON2   0x000ff1       data     extern C:\MCC18\v3_39\src\traditional\proc\p18F2620.asm
              INTCON2bits   0x000ff1       data     extern C:\MCC18\v3_39\src\traditional\proc\p18F2620.asm
                  INTCON3   0x000ff0       data     extern C:\MCC18\v3_39\src\traditional\proc\p18F2620.asm
              INTCON3bits   0x000ff0       data     extern C:\MCC18\v3_39\src\traditional\proc\p18F2620.asm
               INTCONbits   0x000ff2       data     extern C:\MCC18\v3_39\src\traditional\proc\p18F2620.asm
                     IPR1   0x000f9f       data     extern C:\MCC18\v3_39\src\traditional\proc\p18F2620.asm
                 IPR1bits   0x000f9f       data     extern C:\MCC18\v3_39\src\traditional\proc\p18F2620.asm
                     IPR2   0x000fa2       data     extern C:\MCC18\v3_39\src\traditional\proc\p18F2620.asm
                 IPR2bits   0x000fa2       data     extern C:\MCC18\v3_39\src\traditional\proc\p18F2620.asm
                     LATA   0x000f89       data     extern C:\MCC18\v3_39\src\traditional\proc\p18F2620.asm
                 LATAbits   0x000f89       data     extern C:\MCC18\v3_39\src\traditional\proc\p18F2620.asm
                     LATB   0x000f8a       data     extern C:\MCC18\v3_39\src\traditional\proc\p18F2620.asm
                 LATBbits   0x000f8a       data     extern C:\MCC18\v3_39\src\traditional\proc\p18F2620.asm
                     LATC   0x000f8b       data     extern C:\MCC18\v3_39\src\traditional\proc\p18F2620.asm
                 LATCbits   0x000f8b       data     extern C:\MCC18\v3_39\src\traditional\proc\p18F2620.asm
                   LVDCON   0x000fd2       data     extern C:\MCC18\v3_39\src\traditional\proc\p18F2620.asm
               LVDCONbits   0x000fd2       data     extern C:\MCC18\v3_39\src\traditional\proc\p18F2620.asm
                     MyIP   0x000096       data     extern C:\Documents and Settings\User\Desktop\RFID Ethernet\Seconda Parte\Interfaccia Ethernet con ENC28J60\02_icmp_C18\ip.c
                   OSCCON   0x000fd3       data     extern C:\MCC18\v3_39\src\traditional\proc\p18F2620.asm
               OSCCONbits   0x000fd3       data     extern C:\MCC18\v3_39\src\traditional\proc\p18F2620.asm
                  OSCTUNE   0x000f9b       data     extern C:\MCC18\v3_39\src\traditional\proc\p18F2620.asm
              OSCTUNEbits   0x000f9b       data     extern C:\MCC18\v3_39\src\traditional\proc\p18F2620.asm
                       PC   0x000ff9       data     extern C:\MCC18\v3_39\src\traditional\proc\p18F2620.asm
                      PCL   0x000ff9       data     extern C:\MCC18\v3_39\src\traditional\proc\p18F2620.asm
                   PCLATH   0x000ffa       data     extern C:\MCC18\v3_39\src\traditional\proc\p18F2620.asm
                   PCLATU   0x000ffb       data     extern C:\MCC18\v3_39\src\traditional\proc\p18F2620.asm
                     PIE1   0x000f9d       data     extern C:\MCC18\v3_39\src\traditional\proc\p18F2620.asm
                 PIE1bits   0x000f9d       data     extern C:\MCC18\v3_39\src\traditional\proc\p18F2620.asm
                     PIE2   0x000fa0       data     extern C:\MCC18\v3_39\src\traditional\proc\p18F2620.asm
                 PIE2bits   0x000fa0       data     extern C:\MCC18\v3_39\src\traditional\proc\p18F2620.asm
                     PIR1   0x000f9e       data     extern C:\MCC18\v3_39\src\traditional\proc\p18F2620.asm
                 PIR1bits   0x000f9e       data     extern C:\MCC18\v3_39\src\traditional\proc\p18F2620.asm
                     PIR2   0x000fa1       data     extern C:\MCC18\v3_39\src\traditional\proc\p18F2620.asm
                 PIR2bits   0x000fa1       data     extern C:\MCC18\v3_39\src\traditional\proc\p18F2620.asm
                   PLUSW0   0x000feb       data     extern C:\MCC18\v3_39\src\traditional\proc\p18F2620.asm
                   PLUSW1   0x000fe3       data     extern C:\MCC18\v3_39\src\traditional\proc\p18F2620.asm
                   PLUSW2   0x000fdb       data     extern C:\MCC18\v3_39\src\traditional\proc\p18F2620.asm
                    PORTA   0x000f80       data     extern C:\MCC18\v3_39\src\traditional\proc\p18F2620.asm
                PORTAbits   0x000f80       data     extern C:\MCC18\v3_39\src\traditional\proc\p18F2620.asm
                    PORTB   0x000f81       data     extern C:\MCC18\v3_39\src\traditional\proc\p18F2620.asm
                PORTBbits   0x000f81       data     extern C:\MCC18\v3_39\src\traditional\proc\p18F2620.asm
                    PORTC   0x000f82       data     extern C:\MCC18\v3_39\src\traditional\proc\p18F2620.asm
                PORTCbits   0x000f82       data     extern C:\MCC18\v3_39\src\traditional\proc\p18F2620.asm
                    PORTE   0x000f84       data     extern C:\MCC18\v3_39\src\traditional\proc\p18F2620.asm
                PORTEbits   0x000f84       data     extern C:\MCC18\v3_39\src\traditional\proc\p18F2620.asm
                 POSTDEC0   0x000fed       data     extern C:\MCC18\v3_39\src\traditional\proc\p18F2620.asm
                 POSTDEC1   0x000fe5       data     extern C:\MCC18\v3_39\src\traditional\proc\p18F2620.asm
                 POSTDEC2   0x000fdd       data     extern C:\MCC18\v3_39\src\traditional\proc\p18F2620.asm
                 POSTINC0   0x000fee       data     extern C:\MCC18\v3_39\src\traditional\proc\p18F2620.asm
                 POSTINC1   0x000fe6       data     extern C:\MCC18\v3_39\src\traditional\proc\p18F2620.asm
                 POSTINC2   0x000fde       data     extern C:\MCC18\v3_39\src\traditional\proc\p18F2620.asm
                      PR2   0x000fcb       data     extern C:\MCC18\v3_39\src\traditional\proc\p18F2620.asm
                  PREINC0   0x000fec       data     extern C:\MCC18\v3_39\src\traditional\proc\p18F2620.asm
                  PREINC1   0x000fe4       data     extern C:\MCC18\v3_39\src\traditional\proc\p18F2620.asm
                  PREINC2   0x000fdc       data     extern C:\MCC18\v3_39\src\traditional\proc\p18F2620.asm
                     PROD   0x000ff3       data     extern C:\MCC18\v3_39\src\traditional\proc\p18F2620.asm
                    PRODH   0x000ff4       data     extern C:\MCC18\v3_39\src\traditional\proc\p18F2620.asm
                    PRODL   0x000ff3       data     extern C:\MCC18\v3_39\src\traditional\proc\p18F2620.asm
                  PWM1CON   0x000fb7       data     extern C:\MCC18\v3_39\src\traditional\proc\p18F2620.asm
              PWM1CONbits   0x000fb7       data     extern C:\MCC18\v3_39\src\traditional\proc\p18F2620.asm
                     RCON   0x000fd0       data     extern C:\MCC18\v3_39\src\traditional\proc\p18F2620.asm
                 RCONbits   0x000fd0       data     extern C:\MCC18\v3_39\src\traditional\proc\p18F2620.asm
                    RCREG   0x000fae       data     extern C:\MCC18\v3_39\src\traditional\proc\p18F2620.asm
                    RCSTA   0x000fab       data     extern C:\MCC18\v3_39\src\traditional\proc\p18F2620.asm
                RCSTAbits   0x000fab       data     extern C:\MCC18\v3_39\src\traditional\proc\p18F2620.asm
                     RdPt   0x000092       data     extern C:\Documents and Settings\User\Desktop\RFID Ethernet\Seconda Parte\Interfaccia Ethernet con ENC28J60\02_icmp_C18\enc28j60.c
                     SIGN   0x000009       data     extern C:\MCC18\v3_39\src\traditional\math\cmath18.asm
                    SPBRG   0x000faf       data     extern C:\MCC18\v3_39\src\traditional\proc\p18F2620.asm
                   SPBRGH   0x000fb0       data     extern C:\MCC18\v3_39\src\traditional\proc\p18F2620.asm
                   SSPADD   0x000fc8       data     extern C:\MCC18\v3_39\src\traditional\proc\p18F2620.asm
                   SSPBUF   0x000fc9       data     extern C:\MCC18\v3_39\src\traditional\proc\p18F2620.asm
                  SSPCON1   0x000fc6       data     extern C:\MCC18\v3_39\src\traditional\proc\p18F2620.asm
              SSPCON1bits   0x000fc6       data     extern C:\MCC18\v3_39\src\traditional\proc\p18F2620.asm
                  SSPCON2   0x000fc5       data     extern C:\MCC18\v3_39\src\traditional\proc\p18F2620.asm
              SSPCON2bits   0x000fc5       data     extern C:\MCC18\v3_39\src\traditional\proc\p18F2620.asm
                  SSPSTAT   0x000fc7       data     extern C:\MCC18\v3_39\src\traditional\proc\p18F2620.asm
              SSPSTATbits   0x000fc7       data     extern C:\MCC18\v3_39\src\traditional\proc\p18F2620.asm
                   STATUS   0x000fd8       data     extern C:\MCC18\v3_39\src\traditional\proc\p18F2620.asm
               STATUSbits   0x000fd8       data     extern C:\MCC18\v3_39\src\traditional\proc\p18F2620.asm
                   STKPTR   0x000ffc       data     extern C:\MCC18\v3_39\src\traditional\proc\p18F2620.asm
               STKPTRbits   0x000ffc       data     extern C:\MCC18\v3_39\src\traditional\proc\p18F2620.asm
                    T0CON   0x000fd5       data     extern C:\MCC18\v3_39\src\traditional\proc\p18F2620.asm
                T0CONbits   0x000fd5       data     extern C:\MCC18\v3_39\src\traditional\proc\p18F2620.asm
                    T1CON   0x000fcd       data     extern C:\MCC18\v3_39\src\traditional\proc\p18F2620.asm
                T1CONbits   0x000fcd       data     extern C:\MCC18\v3_39\src\traditional\proc\p18F2620.asm
                    T2CON   0x000fca       data     extern C:\MCC18\v3_39\src\traditional\proc\p18F2620.asm
                T2CONbits   0x000fca       data     extern C:\MCC18\v3_39\src\traditional\proc\p18F2620.asm
                    T3CON   0x000fb1       data     extern C:\MCC18\v3_39\src\traditional\proc\p18F2620.asm
                T3CONbits   0x000fb1       data     extern C:\MCC18\v3_39\src\traditional\proc\p18F2620.asm
                   TABLAT   0x000ff5       data     extern C:\MCC18\v3_39\src\traditional\proc\p18F2620.asm
                   TBLPTR   0x000ff6       data     extern C:\MCC18\v3_39\src\traditional\proc\p18F2620.asm
                  TBLPTRH   0x000ff7       data     extern C:\MCC18\v3_39\src\traditional\proc\p18F2620.asm
                  TBLPTRL   0x000ff6       data     extern C:\MCC18\v3_39\src\traditional\proc\p18F2620.asm
                  TBLPTRU   0x000ff8       data     extern C:\MCC18\v3_39\src\traditional\proc\p18F2620.asm
                    TMR0H   0x000fd7       data     extern C:\MCC18\v3_39\src\traditional\proc\p18F2620.asm
                    TMR0L   0x000fd6       data     extern C:\MCC18\v3_39\src\traditional\proc\p18F2620.asm
                    TMR1H   0x000fcf       data     extern C:\MCC18\v3_39\src\traditional\proc\p18F2620.asm
                    TMR1L   0x000fce       data     extern C:\MCC18\v3_39\src\traditional\proc\p18F2620.asm
                     TMR2   0x000fcc       data     extern C:\MCC18\v3_39\src\traditional\proc\p18F2620.asm
                    TMR3H   0x000fb3       data     extern C:\MCC18\v3_39\src\traditional\proc\p18F2620.asm
                    TMR3L   0x000fb2       data     extern C:\MCC18\v3_39\src\traditional\proc\p18F2620.asm
                      TOS   0x000ffd       data     extern C:\MCC18\v3_39\src\traditional\proc\p18F2620.asm
                     TOSH   0x000ffe       data     extern C:\MCC18\v3_39\src\traditional\proc\p18F2620.asm
                     TOSL   0x000ffd       data     extern C:\MCC18\v3_39\src\traditional\proc\p18F2620.asm
                     TOSU   0x000fff       data     extern C:\MCC18\v3_39\src\traditional\proc\p18F2620.asm
                    TRISA   0x000f92       data     extern C:\MCC18\v3_39\src\traditional\proc\p18F2620.asm
                TRISAbits   0x000f92       data     extern C:\MCC18\v3_39\src\traditional\proc\p18F2620.asm
                    TRISB   0x000f93       data     extern C:\MCC18\v3_39\src\traditional\proc\p18F2620.asm
                TRISBbits   0x000f93       data     extern C:\MCC18\v3_39\src\traditional\proc\p18F2620.asm
                    TRISC   0x000f94       data     extern C:\MCC18\v3_39\src\traditional\proc\p18F2620.asm
                TRISCbits   0x000f94       data     extern C:\MCC18\v3_39\src\traditional\proc\p18F2620.asm
                    TXREG   0x000fad       data     extern C:\MCC18\v3_39\src\traditional\proc\p18F2620.asm
                    TXSTA   0x000fac       data     extern C:\MCC18\v3_39\src\traditional\proc\p18F2620.asm
                TXSTAbits   0x000fac       data     extern C:\MCC18\v3_39\src\traditional\proc\p18F2620.asm
                        W   0x000fe8       data     extern C:\MCC18\v3_39\src\traditional\proc\p18F2620.asm
                   WDTCON   0x000fd1       data     extern C:\MCC18\v3_39\src\traditional\proc\p18F2620.asm
               WDTCONbits   0x000fd1       data     extern C:\MCC18\v3_39\src\traditional\proc\p18F2620.asm
                     WREG   0x000fe8       data     extern C:\MCC18\v3_39\src\traditional\proc\p18F2620.asm
                 __AARGB0   0x000007       data     extern C:\MCC18\v3_39\src\traditional\math\aarg.asm
                 __AARGB1   0x000006       data     extern C:\MCC18\v3_39\src\traditional\math\aarg.asm
                 __AARGB2   0x000005       data     extern C:\MCC18\v3_39\src\traditional\math\aarg.asm
                 __AARGB3   0x000004       data     extern C:\MCC18\v3_39\src\traditional\math\aarg.asm
                 __AARGB4   0x000003       data     extern C:\MCC18\v3_39\src\traditional\math\aarg.asm
                 __AARGB5   0x000002       data     extern C:\MCC18\v3_39\src\traditional\math\aarg.asm
                 __AARGB6   0x000001       data     extern C:\MCC18\v3_39\src\traditional\math\aarg.asm
                 __AARGB7   0x000000       data     extern C:\MCC18\v3_39\src\traditional\math\aarg.asm
                   __AEXP   0x000008       data     extern C:\MCC18\v3_39\src\traditional\math\aarg.asm
                __FPFLAGS   0x00000a       data     extern C:\MCC18\v3_39\src\traditional\math\cmath18.asm
            __FPFLAGSbits   0x00000a       data     extern C:\MCC18\v3_39\src\traditional\math\cmath18.asm
                  __REMB0   0x000003       data     extern C:\MCC18\v3_39\src\traditional\math\aarg.asm
                  __REMB1   0x000002       data     extern C:\MCC18\v3_39\src\traditional\math\aarg.asm
                  __REMB2   0x000001       data     extern C:\MCC18\v3_39\src\traditional\math\aarg.asm
                  __REMB3   0x000000       data     extern C:\MCC18\v3_39\src\traditional\math\aarg.asm
                  __tmp_0   0x00000b       data     static C:\Documents and Settings\User\Desktop\RFID Ethernet\Seconda Parte\Interfaccia Ethernet con ENC28J60\02_icmp_C18\enc28j60.c
                  __tmp_0   0x00000b       data     static C:\Documents and Settings\User\Desktop\RFID Ethernet\Seconda Parte\Interfaccia Ethernet con ENC28J60\02_icmp_C18\utility.c
                  __tmp_0   0x00000b       data     static C:\Documents and Settings\User\Desktop\RFID Ethernet\Seconda Parte\Interfaccia Ethernet con ENC28J60\02_icmp_C18\ip.c
                  __tmp_0   0x00000b       data     static C:\Documents and Settings\User\Desktop\RFID Ethernet\Seconda Parte\Interfaccia Ethernet con ENC28J60\02_icmp_C18\arp.c
                  __tmp_0   0x00000b       data     static C:\Documents and Settings\User\Desktop\RFID Ethernet\Seconda Parte\Interfaccia Ethernet con ENC28J60\02_icmp_C18\icmp.c
                  bufSize   0x000090       data     extern C:\Documents and Settings\User\Desktop\RFID Ethernet\Seconda Parte\Interfaccia Ethernet con ENC28J60\02_icmp_C18\enc28j60.c
                curr_byte   0x000083       data     static C:\MCC18\v3_39\src\traditional\startup\c018i.c
               curr_entry   0x000085       data     static C:\MCC18\v3_39\src\traditional\startup\c018i.c
                 data_ptr   0x000087       data     static C:\MCC18\v3_39\src\traditional\startup\c018i.c
                       id   0x00009a       data     extern C:\Documents and Settings\User\Desktop\RFID Ethernet\Seconda Parte\Interfaccia Ethernet con ENC28J60\02_icmp_C18\ip.c
              packetStart   0x000094       data     extern C:\Documents and Settings\User\Desktop\RFID Ethernet\Seconda Parte\Interfaccia Ethernet con ENC28J60\02_icmp_C18\enc28j60.c
                     prom   0x000080       data     static C:\MCC18\v3_39\src\traditional\startup\c018i.c
               remoteAddr   0x00008a       data     extern C:\Documents and Settings\User\Desktop\RFID Ethernet\Seconda Parte\Interfaccia Ethernet con ENC28J60\02_icmp_C18\stack.c



                              Symbols - Sorted by Address
                     Name    Address   Location    Storage File                     
                ---------  ---------  ---------  --------- ---------                
                   _entry   0x000000    program     extern C:\MCC18\v3_39\src\traditional\startup\c018i.c
       ___return_lbl00000   0x000004    program     static                          
                  encInit   0x000038    program     extern C:\Documents and Settings\User\Desktop\RFID Ethernet\Seconda Parte\Interfaccia Ethernet con ENC28J60\02_icmp_C18\enc28j60.c
              DMAChecksum   0x000246    program     extern C:\Documents and Settings\User\Desktop\RFID Ethernet\Seconda Parte\Interfaccia Ethernet con ENC28J60\02_icmp_C18\enc28j60.c
              putChecksum   0x000422    program     extern C:\Documents and Settings\User\Desktop\RFID Ethernet\Seconda Parte\Interfaccia Ethernet con ENC28J60\02_icmp_C18\enc28j60.c
               encDiscard   0x000536    program     extern C:\Documents and Settings\User\Desktop\RFID Ethernet\Seconda Parte\Interfaccia Ethernet con ENC28J60\02_icmp_C18\enc28j60.c
             MACGetHeader   0x0005d6    program     extern C:\Documents and Settings\User\Desktop\RFID Ethernet\Seconda Parte\Interfaccia Ethernet con ENC28J60\02_icmp_C18\enc28j60.c
              freeRxSpace   0x0006ba    program     extern C:\Documents and Settings\User\Desktop\RFID Ethernet\Seconda Parte\Interfaccia Ethernet con ENC28J60\02_icmp_C18\enc28j60.c
             MACPutHeader   0x000764    program     extern C:\Documents and Settings\User\Desktop\RFID Ethernet\Seconda Parte\Interfaccia Ethernet con ENC28J60\02_icmp_C18\enc28j60.c
                  MACSend   0x000842    program     extern C:\Documents and Settings\User\Desktop\RFID Ethernet\Seconda Parte\Interfaccia Ethernet con ENC28J60\02_icmp_C18\enc28j60.c
              isMACLinked   0x0008cc    program     extern C:\Documents and Settings\User\Desktop\RFID Ethernet\Seconda Parte\Interfaccia Ethernet con ENC28J60\02_icmp_C18\enc28j60.c
              encGetArray   0x0008e4    program     extern C:\Documents and Settings\User\Desktop\RFID Ethernet\Seconda Parte\Interfaccia Ethernet con ENC28J60\02_icmp_C18\enc28j60.c
              encPutArray   0x00093a    program     extern C:\Documents and Settings\User\Desktop\RFID Ethernet\Seconda Parte\Interfaccia Ethernet con ENC28J60\02_icmp_C18\enc28j60.c
             encPutString   0x0009a0    program     extern C:\Documents and Settings\User\Desktop\RFID Ethernet\Seconda Parte\Interfaccia Ethernet con ENC28J60\02_icmp_C18\enc28j60.c
                   encPut   0x0009f4    program     extern C:\Documents and Settings\User\Desktop\RFID Ethernet\Seconda Parte\Interfaccia Ethernet con ENC28J60\02_icmp_C18\enc28j60.c
                   encGet   0x000a22    program     extern C:\Documents and Settings\User\Desktop\RFID Ethernet\Seconda Parte\Interfaccia Ethernet con ENC28J60\02_icmp_C18\enc28j60.c
                sendReset   0x000a4e    program     extern C:\Documents and Settings\User\Desktop\RFID Ethernet\Seconda Parte\Interfaccia Ethernet con ENC28J60\02_icmp_C18\enc28j60.c
                 writeReg   0x000a5a    program     extern C:\Documents and Settings\User\Desktop\RFID Ethernet\Seconda Parte\Interfaccia Ethernet con ENC28J60\02_icmp_C18\enc28j60.c
                 writePHY   0x000a84    program     extern C:\Documents and Settings\User\Desktop\RFID Ethernet\Seconda Parte\Interfaccia Ethernet con ENC28J60\02_icmp_C18\enc28j60.c
                  readPHY   0x000b06    program     extern C:\Documents and Settings\User\Desktop\RFID Ethernet\Seconda Parte\Interfaccia Ethernet con ENC28J60\02_icmp_C18\enc28j60.c
                  readMAC   0x000b96    program     extern C:\Documents and Settings\User\Desktop\RFID Ethernet\Seconda Parte\Interfaccia Ethernet con ENC28J60\02_icmp_C18\enc28j60.c
                  readETH   0x000bca    program     extern C:\Documents and Settings\User\Desktop\RFID Ethernet\Seconda Parte\Interfaccia Ethernet con ENC28J60\02_icmp_C18\enc28j60.c
                   BFCReg   0x000bf8    program     extern C:\Documents and Settings\User\Desktop\RFID Ethernet\Seconda Parte\Interfaccia Ethernet con ENC28J60\02_icmp_C18\enc28j60.c
                   BFSReg   0x000c22    program     extern C:\Documents and Settings\User\Desktop\RFID Ethernet\Seconda Parte\Interfaccia Ethernet con ENC28J60\02_icmp_C18\enc28j60.c
                  setBank   0x000c4c    program     extern C:\Documents and Settings\User\Desktop\RFID Ethernet\Seconda Parte\Interfaccia Ethernet con ENC28J60\02_icmp_C18\enc28j60.c
                    spiRW   0x000c7a    program     extern C:\Documents and Settings\User\Desktop\RFID Ethernet\Seconda Parte\Interfaccia Ethernet con ENC28J60\02_icmp_C18\enc28j60.c
                  ipMatch   0x000c9a    program     extern C:\Documents and Settings\User\Desktop\RFID Ethernet\Seconda Parte\Interfaccia Ethernet con ENC28J60\02_icmp_C18\ip.c
             swapIPHeader   0x000cea    program     extern C:\Documents and Settings\User\Desktop\RFID Ethernet\Seconda Parte\Interfaccia Ethernet con ENC28J60\02_icmp_C18\ip.c
                processIP   0x000dd2    program     extern C:\Documents and Settings\User\Desktop\RFID Ethernet\Seconda Parte\Interfaccia Ethernet con ENC28J60\02_icmp_C18\ip.c
              IPPutHeader   0x000f1a    program     extern C:\Documents and Settings\User\Desktop\RFID Ethernet\Seconda Parte\Interfaccia Ethernet con ENC28J60\02_icmp_C18\ip.c
               processARP   0x00108c    program     extern C:\Documents and Settings\User\Desktop\RFID Ethernet\Seconda Parte\Interfaccia Ethernet con ENC28J60\02_icmp_C18\arp.c
              processICMP   0x00125e    program     extern C:\Documents and Settings\User\Desktop\RFID Ethernet\Seconda Parte\Interfaccia Ethernet con ENC28J60\02_icmp_C18\icmp.c
            processPacket   0x001376    program     extern C:\Documents and Settings\User\Desktop\RFID Ethernet\Seconda Parte\Interfaccia Ethernet con ENC28J60\02_icmp_C18\stack.c
                _do_cinit   0x00141c    program     extern C:\MCC18\v3_39\src\traditional\startup\c018i.c
                     test   0x001436    program     static                          
                copy_loop   0x00148e    program     static                          
            copy_one_byte   0x001494    program     static                          
             done_copying   0x0014a2    program     static                          
                     done   0x0014b8    program     static                          
       ___return_lbl00002   0x0014b8    program     static                          
                    htons   0x0014ba    program     extern C:\Documents and Settings\User\Desktop\RFID Ethernet\Seconda Parte\Interfaccia Ethernet con ENC28J60\02_icmp_C18\utility.c
            __zero_memory   0x001504    program     extern C:\MCC18\v3_39\src\traditional\proc\p18F2620.asm
               zero_block   0x001512    program     static C:\MCC18\v3_39\src\traditional\proc\p18F2620.asm
                   loop_h   0x001512    program     static C:\MCC18\v3_39\src\traditional\proc\p18F2620.asm
                compare_l   0x00151a    program     static C:\MCC18\v3_39\src\traditional\proc\p18F2620.asm
                   loop_l   0x00151c    program     static C:\MCC18\v3_39\src\traditional\proc\p18F2620.asm
                 _startup   0x001524    program     extern C:\MCC18\v3_39\src\traditional\startup\c018i.c
                     loop   0x001534    program     static                          
       ___return_lbl00001   0x00153e    program     static                          
             Delay100TCYx   0x001540    program     extern C:\MCC18\v3_39\src\traditional\delays\d100tcyx.asm
       _D100TCYXCODE_0008   0x001548    program     static C:\MCC18\v3_39\src\traditional\delays\d100tcyx.asm
                    D100x   0x00154c    program     static C:\MCC18\v3_39\src\traditional\delays\d100tcyx.asm
                   D100_1   0x00154e    program     static C:\MCC18\v3_39\src\traditional\delays\d100tcyx.asm
       _D100TCYXCODE_0012   0x001552    program     static C:\MCC18\v3_39\src\traditional\delays\d100tcyx.asm
       _D100TCYXCODE_0018   0x001558    program     static C:\MCC18\v3_39\src\traditional\delays\d100tcyx.asm
                     main   0x00155c    program     extern C:\Documents and Settings\User\Desktop\RFID Ethernet\Seconda Parte\Interfaccia Ethernet con ENC28J60\02_icmp_C18\main.c
                   __init   0x001568    program     extern C:\MCC18\v3_39\src\traditional\stdclib\__init.c
               __config_0   0x300001    program     static C:\Documents and Settings\User\Desktop\RFID Ethernet\Seconda Parte\Interfaccia Ethernet con ENC28J60\02_icmp_C18\main.c
               __config_1   0x300002    program     static C:\Documents and Settings\User\Desktop\RFID Ethernet\Seconda Parte\Interfaccia Ethernet con ENC28J60\02_icmp_C18\main.c
               __config_2   0x300003    program     static C:\Documents and Settings\User\Desktop\RFID Ethernet\Seconda Parte\Interfaccia Ethernet con ENC28J60\02_icmp_C18\main.c
               __config_3   0x300005    program     static C:\Documents and Settings\User\Desktop\RFID Ethernet\Seconda Parte\Interfaccia Ethernet con ENC28J60\02_icmp_C18\main.c
               __config_4   0x300006    program     static C:\Documents and Settings\User\Desktop\RFID Ethernet\Seconda Parte\Interfaccia Ethernet con ENC28J60\02_icmp_C18\main.c
                 __AARGB7   0x000000       data     extern C:\MCC18\v3_39\src\traditional\math\aarg.asm
                  __REMB3   0x000000       data     extern C:\MCC18\v3_39\src\traditional\math\aarg.asm
                 __AARGB6   0x000001       data     extern C:\MCC18\v3_39\src\traditional\math\aarg.asm
                  __REMB2   0x000001       data     extern C:\MCC18\v3_39\src\traditional\math\aarg.asm
                 __AARGB5   0x000002       data     extern C:\MCC18\v3_39\src\traditional\math\aarg.asm
                  __REMB1   0x000002       data     extern C:\MCC18\v3_39\src\traditional\math\aarg.asm
                 __AARGB4   0x000003       data     extern C:\MCC18\v3_39\src\traditional\math\aarg.asm
                  __REMB0   0x000003       data     extern C:\MCC18\v3_39\src\traditional\math\aarg.asm
                 __AARGB3   0x000004       data     extern C:\MCC18\v3_39\src\traditional\math\aarg.asm
                 __AARGB2   0x000005       data     extern C:\MCC18\v3_39\src\traditional\math\aarg.asm
                 __AARGB1   0x000006       data     extern C:\MCC18\v3_39\src\traditional\math\aarg.asm
                 __AARGB0   0x000007       data     extern C:\MCC18\v3_39\src\traditional\math\aarg.asm
                   __AEXP   0x000008       data     extern C:\MCC18\v3_39\src\traditional\math\aarg.asm
                     SIGN   0x000009       data     extern C:\MCC18\v3_39\src\traditional\math\cmath18.asm
            __FPFLAGSbits   0x00000a       data     extern C:\MCC18\v3_39\src\traditional\math\cmath18.asm
                __FPFLAGS   0x00000a       data     extern C:\MCC18\v3_39\src\traditional\math\cmath18.asm
                  __tmp_0   0x00000b       data     static C:\Documents and Settings\User\Desktop\RFID Ethernet\Seconda Parte\Interfaccia Ethernet con ENC28J60\02_icmp_C18\ip.c
                  __tmp_0   0x00000b       data     static C:\Documents and Settings\User\Desktop\RFID Ethernet\Seconda Parte\Interfaccia Ethernet con ENC28J60\02_icmp_C18\utility.c
                  __tmp_0   0x00000b       data     static C:\Documents and Settings\User\Desktop\RFID Ethernet\Seconda Parte\Interfaccia Ethernet con ENC28J60\02_icmp_C18\enc28j60.c
                  __tmp_0   0x00000b       data     static C:\Documents and Settings\User\Desktop\RFID Ethernet\Seconda Parte\Interfaccia Ethernet con ENC28J60\02_icmp_C18\arp.c
                  __tmp_0   0x00000b       data     static C:\Documents and Settings\User\Desktop\RFID Ethernet\Seconda Parte\Interfaccia Ethernet con ENC28J60\02_icmp_C18\icmp.c
            DelayCounter1   0x000011       data     extern C:\MCC18\v3_39\src\traditional\delays\delayd1.asm
                     prom   0x000080       data     static C:\MCC18\v3_39\src\traditional\startup\c018i.c
                curr_byte   0x000083       data     static C:\MCC18\v3_39\src\traditional\startup\c018i.c
               curr_entry   0x000085       data     static C:\MCC18\v3_39\src\traditional\startup\c018i.c
                 data_ptr   0x000087       data     static C:\MCC18\v3_39\src\traditional\startup\c018i.c
               remoteAddr   0x00008a       data     extern C:\Documents and Settings\User\Desktop\RFID Ethernet\Seconda Parte\Interfaccia Ethernet con ENC28J60\02_icmp_C18\stack.c
                  bufSize   0x000090       data     extern C:\Documents and Settings\User\Desktop\RFID Ethernet\Seconda Parte\Interfaccia Ethernet con ENC28J60\02_icmp_C18\enc28j60.c
                     RdPt   0x000092       data     extern C:\Documents and Settings\User\Desktop\RFID Ethernet\Seconda Parte\Interfaccia Ethernet con ENC28J60\02_icmp_C18\enc28j60.c
              packetStart   0x000094       data     extern C:\Documents and Settings\User\Desktop\RFID Ethernet\Seconda Parte\Interfaccia Ethernet con ENC28J60\02_icmp_C18\enc28j60.c
                     MyIP   0x000096       data     extern C:\Documents and Settings\User\Desktop\RFID Ethernet\Seconda Parte\Interfaccia Ethernet con ENC28J60\02_icmp_C18\ip.c
                       id   0x00009a       data     extern C:\Documents and Settings\User\Desktop\RFID Ethernet\Seconda Parte\Interfaccia Ethernet con ENC28J60\02_icmp_C18\ip.c
                PORTAbits   0x000f80       data     extern C:\MCC18\v3_39\src\traditional\proc\p18F2620.asm
                    PORTA   0x000f80       data     extern C:\MCC18\v3_39\src\traditional\proc\p18F2620.asm
                PORTBbits   0x000f81       data     extern C:\MCC18\v3_39\src\traditional\proc\p18F2620.asm
                    PORTB   0x000f81       data     extern C:\MCC18\v3_39\src\traditional\proc\p18F2620.asm
                PORTCbits   0x000f82       data     extern C:\MCC18\v3_39\src\traditional\proc\p18F2620.asm
                    PORTC   0x000f82       data     extern C:\MCC18\v3_39\src\traditional\proc\p18F2620.asm
                    PORTE   0x000f84       data     extern C:\MCC18\v3_39\src\traditional\proc\p18F2620.asm
                PORTEbits   0x000f84       data     extern C:\MCC18\v3_39\src\traditional\proc\p18F2620.asm
                     LATA   0x000f89       data     extern C:\MCC18\v3_39\src\traditional\proc\p18F2620.asm
                 LATAbits   0x000f89       data     extern C:\MCC18\v3_39\src\traditional\proc\p18F2620.asm
                     LATB   0x000f8a       data     extern C:\MCC18\v3_39\src\traditional\proc\p18F2620.asm
                 LATBbits   0x000f8a       data     extern C:\MCC18\v3_39\src\traditional\proc\p18F2620.asm
                     LATC   0x000f8b       data     extern C:\MCC18\v3_39\src\traditional\proc\p18F2620.asm
                 LATCbits   0x000f8b       data     extern C:\MCC18\v3_39\src\traditional\proc\p18F2620.asm
                 DDRAbits   0x000f92       data     extern C:\MCC18\v3_39\src\traditional\proc\p18F2620.asm
                     DDRA   0x000f92       data     extern C:\MCC18\v3_39\src\traditional\proc\p18F2620.asm
                    TRISA   0x000f92       data     extern C:\MCC18\v3_39\src\traditional\proc\p18F2620.asm
                TRISAbits   0x000f92       data     extern C:\MCC18\v3_39\src\traditional\proc\p18F2620.asm
                 DDRBbits   0x000f93       data     extern C:\MCC18\v3_39\src\traditional\proc\p18F2620.asm
                     DDRB   0x000f93       data     extern C:\MCC18\v3_39\src\traditional\proc\p18F2620.asm
                    TRISB   0x000f93       data     extern C:\MCC18\v3_39\src\traditional\proc\p18F2620.asm
                TRISBbits   0x000f93       data     extern C:\MCC18\v3_39\src\traditional\proc\p18F2620.asm
                    TRISC   0x000f94       data     extern C:\MCC18\v3_39\src\traditional\proc\p18F2620.asm
                TRISCbits   0x000f94       data     extern C:\MCC18\v3_39\src\traditional\proc\p18F2620.asm
                 DDRCbits   0x000f94       data     extern C:\MCC18\v3_39\src\traditional\proc\p18F2620.asm
                     DDRC   0x000f94       data     extern C:\MCC18\v3_39\src\traditional\proc\p18F2620.asm
              OSCTUNEbits   0x000f9b       data     extern C:\MCC18\v3_39\src\traditional\proc\p18F2620.asm
                  OSCTUNE   0x000f9b       data     extern C:\MCC18\v3_39\src\traditional\proc\p18F2620.asm
                     PIE1   0x000f9d       data     extern C:\MCC18\v3_39\src\traditional\proc\p18F2620.asm
                 PIE1bits   0x000f9d       data     extern C:\MCC18\v3_39\src\traditional\proc\p18F2620.asm
                 PIR1bits   0x000f9e       data     extern C:\MCC18\v3_39\src\traditional\proc\p18F2620.asm
                     PIR1   0x000f9e       data     extern C:\MCC18\v3_39\src\traditional\proc\p18F2620.asm
                     IPR1   0x000f9f       data     extern C:\MCC18\v3_39\src\traditional\proc\p18F2620.asm
                 IPR1bits   0x000f9f       data     extern C:\MCC18\v3_39\src\traditional\proc\p18F2620.asm
                 PIE2bits   0x000fa0       data     extern C:\MCC18\v3_39\src\traditional\proc\p18F2620.asm
                     PIE2   0x000fa0       data     extern C:\MCC18\v3_39\src\traditional\proc\p18F2620.asm
                 PIR2bits   0x000fa1       data     extern C:\MCC18\v3_39\src\traditional\proc\p18F2620.asm
                     PIR2   0x000fa1       data     extern C:\MCC18\v3_39\src\traditional\proc\p18F2620.asm
                 IPR2bits   0x000fa2       data     extern C:\MCC18\v3_39\src\traditional\proc\p18F2620.asm
                     IPR2   0x000fa2       data     extern C:\MCC18\v3_39\src\traditional\proc\p18F2620.asm
                   EECON1   0x000fa6       data     extern C:\MCC18\v3_39\src\traditional\proc\p18F2620.asm
               EECON1bits   0x000fa6       data     extern C:\MCC18\v3_39\src\traditional\proc\p18F2620.asm
                   EECON2   0x000fa7       data     extern C:\MCC18\v3_39\src\traditional\proc\p18F2620.asm
                   EEDATA   0x000fa8       data     extern C:\MCC18\v3_39\src\traditional\proc\p18F2620.asm
                    EEADR   0x000fa9       data     extern C:\MCC18\v3_39\src\traditional\proc\p18F2620.asm
                   EEADRH   0x000faa       data     extern C:\MCC18\v3_39\src\traditional\proc\p18F2620.asm
                    RCSTA   0x000fab       data     extern C:\MCC18\v3_39\src\traditional\proc\p18F2620.asm
                RCSTAbits   0x000fab       data     extern C:\MCC18\v3_39\src\traditional\proc\p18F2620.asm
                TXSTAbits   0x000fac       data     extern C:\MCC18\v3_39\src\traditional\proc\p18F2620.asm
                    TXSTA   0x000fac       data     extern C:\MCC18\v3_39\src\traditional\proc\p18F2620.asm
                    TXREG   0x000fad       data     extern C:\MCC18\v3_39\src\traditional\proc\p18F2620.asm
                    RCREG   0x000fae       data     extern C:\MCC18\v3_39\src\traditional\proc\p18F2620.asm
                    SPBRG   0x000faf       data     extern C:\MCC18\v3_39\src\traditional\proc\p18F2620.asm
                   SPBRGH   0x000fb0       data     extern C:\MCC18\v3_39\src\traditional\proc\p18F2620.asm
                    T3CON   0x000fb1       data     extern C:\MCC18\v3_39\src\traditional\proc\p18F2620.asm
                T3CONbits   0x000fb1       data     extern C:\MCC18\v3_39\src\traditional\proc\p18F2620.asm
                    TMR3L   0x000fb2       data     extern C:\MCC18\v3_39\src\traditional\proc\p18F2620.asm
                    TMR3H   0x000fb3       data     extern C:\MCC18\v3_39\src\traditional\proc\p18F2620.asm
                CMCONbits   0x000fb4       data     extern C:\MCC18\v3_39\src\traditional\proc\p18F2620.asm
                    CMCON   0x000fb4       data     extern C:\MCC18\v3_39\src\traditional\proc\p18F2620.asm
                   CVRCON   0x000fb5       data     extern C:\MCC18\v3_39\src\traditional\proc\p18F2620.asm
               CVRCONbits   0x000fb5       data     extern C:\MCC18\v3_39\src\traditional\proc\p18F2620.asm
              ECCP1ASbits   0x000fb6       data     extern C:\MCC18\v3_39\src\traditional\proc\p18F2620.asm
                  ECCP1AS   0x000fb6       data     extern C:\MCC18\v3_39\src\traditional\proc\p18F2620.asm
               ECCPASbits   0x000fb6       data     extern C:\MCC18\v3_39\src\traditional\proc\p18F2620.asm
                   ECCPAS   0x000fb6       data     extern C:\MCC18\v3_39\src\traditional\proc\p18F2620.asm
                  PWM1CON   0x000fb7       data     extern C:\MCC18\v3_39\src\traditional\proc\p18F2620.asm
              PWM1CONbits   0x000fb7       data     extern C:\MCC18\v3_39\src\traditional\proc\p18F2620.asm
             ECCP1DELbits   0x000fb7       data     extern C:\MCC18\v3_39\src\traditional\proc\p18F2620.asm
                 ECCP1DEL   0x000fb7       data     extern C:\MCC18\v3_39\src\traditional\proc\p18F2620.asm
                  BAUDCON   0x000fb8       data     extern C:\MCC18\v3_39\src\traditional\proc\p18F2620.asm
              BAUDCONbits   0x000fb8       data     extern C:\MCC18\v3_39\src\traditional\proc\p18F2620.asm
                  BAUDCTL   0x000fb8       data     extern C:\MCC18\v3_39\src\traditional\proc\p18F2620.asm
              BAUDCTLbits   0x000fb8       data     extern C:\MCC18\v3_39\src\traditional\proc\p18F2620.asm
              CCP2CONbits   0x000fba       data     extern C:\MCC18\v3_39\src\traditional\proc\p18F2620.asm
                  CCP2CON   0x000fba       data     extern C:\MCC18\v3_39\src\traditional\proc\p18F2620.asm
                    CCPR2   0x000fbb       data     extern C:\MCC18\v3_39\src\traditional\proc\p18F2620.asm
                   CCPR2L   0x000fbb       data     extern C:\MCC18\v3_39\src\traditional\proc\p18F2620.asm
                   CCPR2H   0x000fbc       data     extern C:\MCC18\v3_39\src\traditional\proc\p18F2620.asm
              CCP1CONbits   0x000fbd       data     extern C:\MCC18\v3_39\src\traditional\proc\p18F2620.asm
                  CCP1CON   0x000fbd       data     extern C:\MCC18\v3_39\src\traditional\proc\p18F2620.asm
                    CCPR1   0x000fbe       data     extern C:\MCC18\v3_39\src\traditional\proc\p18F2620.asm
                   CCPR1L   0x000fbe       data     extern C:\MCC18\v3_39\src\traditional\proc\p18F2620.asm
                   CCPR1H   0x000fbf       data     extern C:\MCC18\v3_39\src\traditional\proc\p18F2620.asm
               ADCON2bits   0x000fc0       data     extern C:\MCC18\v3_39\src\traditional\proc\p18F2620.asm
                   ADCON2   0x000fc0       data     extern C:\MCC18\v3_39\src\traditional\proc\p18F2620.asm
               ADCON1bits   0x000fc1       data     extern C:\MCC18\v3_39\src\traditional\proc\p18F2620.asm
                   ADCON1   0x000fc1       data     extern C:\MCC18\v3_39\src\traditional\proc\p18F2620.asm
               ADCON0bits   0x000fc2       data     extern C:\MCC18\v3_39\src\traditional\proc\p18F2620.asm
                   ADCON0   0x000fc2       data     extern C:\MCC18\v3_39\src\traditional\proc\p18F2620.asm
                    ADRES   0x000fc3       data     extern C:\MCC18\v3_39\src\traditional\proc\p18F2620.asm
                   ADRESL   0x000fc3       data     extern C:\MCC18\v3_39\src\traditional\proc\p18F2620.asm
                   ADRESH   0x000fc4       data     extern C:\MCC18\v3_39\src\traditional\proc\p18F2620.asm
              SSPCON2bits   0x000fc5       data     extern C:\MCC18\v3_39\src\traditional\proc\p18F2620.asm
                  SSPCON2   0x000fc5       data     extern C:\MCC18\v3_39\src\traditional\proc\p18F2620.asm
                  SSPCON1   0x000fc6       data     extern C:\MCC18\v3_39\src\traditional\proc\p18F2620.asm
              SSPCON1bits   0x000fc6       data     extern C:\MCC18\v3_39\src\traditional\proc\p18F2620.asm
              SSPSTATbits   0x000fc7       data     extern C:\MCC18\v3_39\src\traditional\proc\p18F2620.asm
                  SSPSTAT   0x000fc7       data     extern C:\MCC18\v3_39\src\traditional\proc\p18F2620.asm
                   SSPADD   0x000fc8       data     extern C:\MCC18\v3_39\src\traditional\proc\p18F2620.asm
                   SSPBUF   0x000fc9       data     extern C:\MCC18\v3_39\src\traditional\proc\p18F2620.asm
                    T2CON   0x000fca       data     extern C:\MCC18\v3_39\src\traditional\proc\p18F2620.asm
                T2CONbits   0x000fca       data     extern C:\MCC18\v3_39\src\traditional\proc\p18F2620.asm
                      PR2   0x000fcb       data     extern C:\MCC18\v3_39\src\traditional\proc\p18F2620.asm
                     TMR2   0x000fcc       data     extern C:\MCC18\v3_39\src\traditional\proc\p18F2620.asm
                T1CONbits   0x000fcd       data     extern C:\MCC18\v3_39\src\traditional\proc\p18F2620.asm
                    T1CON   0x000fcd       data     extern C:\MCC18\v3_39\src\traditional\proc\p18F2620.asm
                    TMR1L   0x000fce       data     extern C:\MCC18\v3_39\src\traditional\proc\p18F2620.asm
                    TMR1H   0x000fcf       data     extern C:\MCC18\v3_39\src\traditional\proc\p18F2620.asm
                 RCONbits   0x000fd0       data     extern C:\MCC18\v3_39\src\traditional\proc\p18F2620.asm
                     RCON   0x000fd0       data     extern C:\MCC18\v3_39\src\traditional\proc\p18F2620.asm
               WDTCONbits   0x000fd1       data     extern C:\MCC18\v3_39\src\traditional\proc\p18F2620.asm
                   WDTCON   0x000fd1       data     extern C:\MCC18\v3_39\src\traditional\proc\p18F2620.asm
               LVDCONbits   0x000fd2       data     extern C:\MCC18\v3_39\src\traditional\proc\p18F2620.asm
                   LVDCON   0x000fd2       data     extern C:\MCC18\v3_39\src\traditional\proc\p18F2620.asm
              HLVDCONbits   0x000fd2       data     extern C:\MCC18\v3_39\src\traditional\proc\p18F2620.asm
                  HLVDCON   0x000fd2       data     extern C:\MCC18\v3_39\src\traditional\proc\p18F2620.asm
               OSCCONbits   0x000fd3       data     extern C:\MCC18\v3_39\src\traditional\proc\p18F2620.asm
                   OSCCON   0x000fd3       data     extern C:\MCC18\v3_39\src\traditional\proc\p18F2620.asm
                T0CONbits   0x000fd5       data     extern C:\MCC18\v3_39\src\traditional\proc\p18F2620.asm
                    T0CON   0x000fd5       data     extern C:\MCC18\v3_39\src\traditional\proc\p18F2620.asm
                    TMR0L   0x000fd6       data     extern C:\MCC18\v3_39\src\traditional\proc\p18F2620.asm
                    TMR0H   0x000fd7       data     extern C:\MCC18\v3_39\src\traditional\proc\p18F2620.asm
                   STATUS   0x000fd8       data     extern C:\MCC18\v3_39\src\traditional\proc\p18F2620.asm
               STATUSbits   0x000fd8       data     extern C:\MCC18\v3_39\src\traditional\proc\p18F2620.asm
                     FSR2   0x000fd9       data     extern C:\MCC18\v3_39\src\traditional\proc\p18F2620.asm
                    FSR2L   0x000fd9       data     extern C:\MCC18\v3_39\src\traditional\proc\p18F2620.asm
                    FSR2H   0x000fda       data     extern C:\MCC18\v3_39\src\traditional\proc\p18F2620.asm
                   PLUSW2   0x000fdb       data     extern C:\MCC18\v3_39\src\traditional\proc\p18F2620.asm
                  PREINC2   0x000fdc       data     extern C:\MCC18\v3_39\src\traditional\proc\p18F2620.asm
                 POSTDEC2   0x000fdd       data     extern C:\MCC18\v3_39\src\traditional\proc\p18F2620.asm
                 POSTINC2   0x000fde       data     extern C:\MCC18\v3_39\src\traditional\proc\p18F2620.asm
                    INDF2   0x000fdf       data     extern C:\MCC18\v3_39\src\traditional\proc\p18F2620.asm
                      BSR   0x000fe0       data     extern C:\MCC18\v3_39\src\traditional\proc\p18F2620.asm
                     FSR1   0x000fe1       data     extern C:\MCC18\v3_39\src\traditional\proc\p18F2620.asm
                    FSR1L   0x000fe1       data     extern C:\MCC18\v3_39\src\traditional\proc\p18F2620.asm
                    FSR1H   0x000fe2       data     extern C:\MCC18\v3_39\src\traditional\proc\p18F2620.asm
                   PLUSW1   0x000fe3       data     extern C:\MCC18\v3_39\src\traditional\proc\p18F2620.asm
                  PREINC1   0x000fe4       data     extern C:\MCC18\v3_39\src\traditional\proc\p18F2620.asm
                 POSTDEC1   0x000fe5       data     extern C:\MCC18\v3_39\src\traditional\proc\p18F2620.asm
                 POSTINC1   0x000fe6       data     extern C:\MCC18\v3_39\src\traditional\proc\p18F2620.asm
                    INDF1   0x000fe7       data     extern C:\MCC18\v3_39\src\traditional\proc\p18F2620.asm
                     WREG   0x000fe8       data     extern C:\MCC18\v3_39\src\traditional\proc\p18F2620.asm
                        W   0x000fe8       data     extern C:\MCC18\v3_39\src\traditional\proc\p18F2620.asm
                    FSR0L   0x000fe9       data     extern C:\MCC18\v3_39\src\traditional\proc\p18F2620.asm
                     FSR0   0x000fe9       data     extern C:\MCC18\v3_39\src\traditional\proc\p18F2620.asm
                    FSR0H   0x000fea       data     extern C:\MCC18\v3_39\src\traditional\proc\p18F2620.asm
                   PLUSW0   0x000feb       data     extern C:\MCC18\v3_39\src\traditional\proc\p18F2620.asm
                  PREINC0   0x000fec       data     extern C:\MCC18\v3_39\src\traditional\proc\p18F2620.asm
                 POSTDEC0   0x000fed       data     extern C:\MCC18\v3_39\src\traditional\proc\p18F2620.asm
                 POSTINC0   0x000fee       data     extern C:\MCC18\v3_39\src\traditional\proc\p18F2620.asm
                    INDF0   0x000fef       data     extern C:\MCC18\v3_39\src\traditional\proc\p18F2620.asm
              INTCON3bits   0x000ff0       data     extern C:\MCC18\v3_39\src\traditional\proc\p18F2620.asm
                  INTCON3   0x000ff0       data     extern C:\MCC18\v3_39\src\traditional\proc\p18F2620.asm
              INTCON2bits   0x000ff1       data     extern C:\MCC18\v3_39\src\traditional\proc\p18F2620.asm
                  INTCON2   0x000ff1       data     extern C:\MCC18\v3_39\src\traditional\proc\p18F2620.asm
               INTCONbits   0x000ff2       data     extern C:\MCC18\v3_39\src\traditional\proc\p18F2620.asm
                   INTCON   0x000ff2       data     extern C:\MCC18\v3_39\src\traditional\proc\p18F2620.asm
                     PROD   0x000ff3       data     extern C:\MCC18\v3_39\src\traditional\proc\p18F2620.asm
                    PRODL   0x000ff3       data     extern C:\MCC18\v3_39\src\traditional\proc\p18F2620.asm
                    PRODH   0x000ff4       data     extern C:\MCC18\v3_39\src\traditional\proc\p18F2620.asm
                   TABLAT   0x000ff5       data     extern C:\MCC18\v3_39\src\traditional\proc\p18F2620.asm
                   TBLPTR   0x000ff6       data     extern C:\MCC18\v3_39\src\traditional\proc\p18F2620.asm
                  TBLPTRL   0x000ff6       data     extern C:\MCC18\v3_39\src\traditional\proc\p18F2620.asm
                  TBLPTRH   0x000ff7       data     extern C:\MCC18\v3_39\src\traditional\proc\p18F2620.asm
                  TBLPTRU   0x000ff8       data     extern C:\MCC18\v3_39\src\traditional\proc\p18F2620.asm
                      PCL   0x000ff9       data     extern C:\MCC18\v3_39\src\traditional\proc\p18F2620.asm
                       PC   0x000ff9       data     extern C:\MCC18\v3_39\src\traditional\proc\p18F2620.asm
                   PCLATH   0x000ffa       data     extern C:\MCC18\v3_39\src\traditional\proc\p18F2620.asm
                   PCLATU   0x000ffb       data     extern C:\MCC18\v3_39\src\traditional\proc\p18F2620.asm
               STKPTRbits   0x000ffc       data     extern C:\MCC18\v3_39\src\traditional\proc\p18F2620.asm
                   STKPTR   0x000ffc       data     extern C:\MCC18\v3_39\src\traditional\proc\p18F2620.asm
                      TOS   0x000ffd       data     extern C:\MCC18\v3_39\src\traditional\proc\p18F2620.asm
                     TOSL   0x000ffd       data     extern C:\MCC18\v3_39\src\traditional\proc\p18F2620.asm
                     TOSH   0x000ffe       data     extern C:\MCC18\v3_39\src\traditional\proc\p18F2620.asm
                     TOSU   0x000fff       data     extern C:\MCC18\v3_39\src\traditional\proc\p18F2620.asm


